:100000000C94E0010C9423020C9408020C94080256
:100010000C9408020C9408020C9408020C94A10D94
:100020000C9408020C9408020C9408020C94080228
:100030000C9408020C944E050C9408020C940802CF
:100040000C94EC0A0C9408020C9408020C9408021C
:100050000C9408020C9408020C9408020C940802F8
:100060000C9408020C940802040309042003720093
:1000700061006E006300690064006200610063005B
:100080006F006E002E0063006F006D0018035500B6
:10009000730062004B006500790062006F00610030
:1000A000720064001201100100000008424231E1B8
:1000B0000001010200010902220001010080320951
:1000C00004000001030000000921010100012223B6
:1000D000000705810308000A05010906A1010507BB
:1000E00019E029E71500250175019508810295039E
:1000F00075082565190029658100C02C001E013492
:1001000001200121012201240134012601270125BA
:10011000012E0136002D003700380027001E001F79
:1001200000200021002200230024002500260033A7
:1001300000330136012E00370138011F010400058C
:100140000006000700080009000A000B000C000D63
:10015000000E000F00100011001200130014001513
:100160000016001700180019001A001B001C001DC3
:10017000001F02220227022C023002320237023B09
:10018000024002430248024C025102540257025BF1
:10019000026002650269026D026F02730278027CDE
:1001A00002810286028B02910297029D02A302A99C
:1001B00002AF02B502BB02C102C702CE02D502DC09
:1001C00002E302EA02F002F602FD0203030A03114F
:1001D0000317031D0324032B0332033A0341034A8D
:1001E00003500357036162636465666768696A6BFD
:1001F0006C6D6E6F707172737475767778797A3012
:100200003132333435363738392E2C3F27212F28D9
:1002100029263A3B3D2B2D5F222440080A0A072E4F
:100220002D002D2E2E2E002D2E2D2E002D2E2E00AB
:100230002E002E2E2D2E002D2D2E002E2E2E2E0099
:100240002E2E002E2D2D2D002D2E2D002E2D2E2E5E
:10025000002D2D002D2E002D2D2D002E2D2D2E00AC
:100260002D2D2E2D002E2D2E002E2E2E002D002E6B
:100270002E2D002E2E2E2D002E2D2D002D2E2E2D2E
:10028000002D2E2D2D002D2D2E2E002D2D2D2D2D22
:10029000002E2D2D2D2D002E2E2D2D2D002E2E2E0F
:1002A0002D2D002E2E2E2E2D002E2E2E2E2E002DFC
:1002B0002E2E2E2E002D2D2E2E2E002D2D2D2E2EBF
:1002C000002D2D2D2D2E002E2D2E2D2E2D002D2DE1
:1002D0002E2E2D2D002E2E2D2D2E2E002E2D2D2DA1
:1002E0002D2E002D2E2D2E2D2D002D2E2E2D2E00BF
:1002F0002D2E2D2D2E002D2E2D2D2E2D002E2D2E82
:100300002E2E002D2D2D2E2E2E002D2E2D2E2D2E6F
:10031000002D2E2E2E2D002E2D2E2D2E002D2E2E8C
:100320002E2E2D002E2E2D2D2E2D002E2D2E2E2D4F
:100330002E002E2E2E2D2E2E2D002E2D2D2E2D2E3E
:10034000002E2E2E2E2E2E2E2E002D2E2D2E2D005A
:100350002E2E2E2D2E2D002E2E2E2D2D2D2E2E2EF0
:10036000000200000000240027002A000000000016
:10037000250028002B000000000023002600290093
:10038000040404040404040402020202020203033B
:100390000303030301020408102040800102040843
:1003A00010200102040810200000000700020100D4
:1003B0000003040600000000000000004905500A88
:1003C00011241FBECFEFD4E0DEBFCDBF12E0A0E00E
:1003D000B1E0EAE9F3E202C005900D92AA32B1075A
:1003E000D9F713E0AAE2B2E001C01D92A330B10731
:1003F000E1F713E0C0ECD3E004C02297FE010E94B5
:10040000C711CC3BD107C9F70E9429100C94CB111E
:100410000C940000A82FB92F80E090E041E050EA52
:10042000609530E009C02D9182279795879510F04F
:1004300084279527305EC8F36F5FA8F30895EADF3D
:100440008D939D930895CF93CFB7CF93DF93C395AB
:100450004B9BE9F74B9B0BC04B9B09C04B9B07C0C9
:100460004B9B05C04B9B03C04B9B01C08BC06F9344
:10047000C091E602DD27C351DD4F2F9365E54B9B0D
:1004800003C02F916F91E6CF0F931F934F9320E0FE
:1004900040E15F9309B10C7003FB27F93F9350E0F3
:1004A0003BE039C01C7040642F77012F5F5F1EC096
:1004B000406819B11C702F7752501FC0406409B1B9
:1004C0002F770C70D1F15F5F00C023C0406219B17B
:1004D0002F771C7091F15F5F00C025C00C70102752
:1004E000515012F45D5F0000115027952C3F19B157
:1004F000C8F61C700127015027952C3FC8F64227EB
:10050000499309B10C7010274F73115027952C3F58
:10051000A8F64695469519B11C7079F0012701504F
:1005200027952C3F98F66B5A60F3315009B1B0F61D
:1005300000C011E01CBB002719C03B503195C31B04
:10054000D04011E01CBB0881033C09F10B34F9F0E9
:100550002091E4021981110F1213EDCF4A81441F3B
:10056000093651F10D3211F0013E29F70093EB02EB
:100570003F915F914F911F910F912F916F91CCB34C
:10058000C0FD65CFDF91CF91CFBFCF91189520915E
:10059000EB02222369F31091E902112391F5343023
:1005A00092F13093E9022093E5021091E6023BE0DC
:1005B000311B3093E60227C00091E90201300CF5AF
:1005C0000AE54F7049F43091040234FD1DC00093D8
:1005D0000402CDECD2E01CC03091D80234FD14C02E
:1005E0000093D802C9EDD2E013C0052710E000C087
:1005F00000000BB91AC0052710E0221F1DC010E033
:1006000021C04AE502C032ED432FC4E1D0E032E020
:100610001AB11C605B9A0BB11AB95CE020E865E383
:1006200020FF05270BB9279517951C3FF0F6669517
:10063000B8F7B1F720FF05270BB9279517951C3F91
:10064000D0F62795179517FF052700001C3F0BB91B
:10065000B0F629913A9519F7037F1091EA02110F2C
:10066000C651D0400BB911F01093E40211E01CBB4D
:1006700008601AB1137F402F437F54E05A95F1F779
:100680000BB91AB94BB974CFFB01DC0105900D927F
:100690000020E1F70895FB01DC018D9101908019A4
:1006A0000110D9F3990B0895F999FECF72BD61BD80
:1006B000F89A80B50895F999FECF1FBA72BD61BD51
:1006C00040BD0FB6F894FA9AF99A0FBE0895E9E67C
:1006D000F0E0808182608083E89A8BE48093D90285
:1006E0008AE58093D80208951F93CF93DF9390916A
:1006F000E902935097FDAAC02091E6028091E5029D
:100700008D3209F0A1C0983009F09EC0CCE0D0E055
:10071000C21BD109C351DD4F83EC8093CD028AE522
:100720008093040210922B028881807629F0CE01FA
:100730000E94A504282F7FC09A811092D602898139
:10074000882331F41092D70286ED92E022E06FC048
:10075000853019F49093EA0267C0863009F04FC0E3
:100760008B81813041F484EA90E09093E802809399
:10077000E70222E140C0823041F486EB90E09093A2
:10078000E8028093E70222E236C08330F9F48A81DE
:10079000882341F488E690E09093E8028093E70292
:1007A00024E029C0813041F48CE690E09093E80287
:1007B0008093E70220E21FC08230E1F48CE890E0F1
:1007C0009093E8028093E70228E115C0813241F45A
:1007D00088EC90E09093E8028093E70229E00BC058
:1007E000823241F488ED90E09093E8028093E70232
:1007F00023E201C020E080E480932B021CC08830FB
:1008000019F48CEE92E009C0893019F49093EC024F
:100810000BC08A3021F486ED92E021E008C08B30D5
:1008200019F48BE48093D90286ED92E020E0909356
:10083000E8028093E7028F81882321F48E8182175A
:1008400008F4282F209305021092E90280910402F7
:1008500084FF4AC0809105028F3F09F445C0182FDC
:10086000893008F018E0811B809305028091CD0249
:1008700098E889278093CD02112341F12091E70266
:100880003091E80280912B0286FF0DC0AEECB2E001
:1008900080E090E0F901E80FF91FE491ED930196F3
:1008A0001817C1F708C0912FD901EEECF2E08D9135
:1008B00081939150E1F71150812F90E01F5F0196D5
:1008C000820F931F9093E8028093E7028EEC92E0F0
:1008D000612F0E941F02612F6C5F6C3019F08FEF47
:1008E000809305026093040294E189B18C7031F425
:1008F0009150D9F71092EA021092E402DF91CF9161
:100900001F9108951F93DC01162F8091D80284FF58
:1009100007C08091D90298E889278093D90203C043
:100920008AE58093D802912FEAEDF2E08D918193D0
:1009300091501916DCF38AED92E0612F0E941F029C
:100940001C5F1093D8021F910895FC018CE292E085
:100950009093E8028093E70280818076803251F4A0
:100960008181813039F0823029F08A3019F4838115
:100970008093320280E008958091D80284FFFCCFFA
:1009800010922C0210922D0210922E0210922F0221
:1009900040932C0260932D028CE292E064E00E946E
:1009A00082048091D80284FFFCCF10922C02109216
:1009B0002D0210922E0210922F028CE292E064E03F
:1009C0000E948204089540E00E94BC0408950E94A1
:1009D000740308959C016A3011F468E232C06830F3
:1009E00011F46AE22EC0862F81548A3148F4E62F32
:1009F000F0E0EE0FFF1FE554FF4F659174911BC0AF
:100A0000862F81568A3148F4E62FF0E0EE0FFF1F63
:100A1000E558FF4F6591749113C06032A0F0E62F46
:100A2000F0E0EE0FFF1FE554FF4F659174916F3FAB
:100A3000710531F02CF0C90142E00E94BC0403C0F2
:100A4000C9010E94E3040E9474030895FC0184E23A
:100A500092E0918380831BB88AB1836F8AB9EEE6F6
:100A6000F0E080811082F89454985C98549A5C9AD3
:100A70000E946703789410922C0210922D0210921B
:100A80002E0210922F028CE292E064E00E94820417
:100A9000089580E392E00E94260508951F920F9228
:100AA0000FB60F9211248F939F93AF93BF937894B7
:100AB0008091560290915702A0915802B09159022C
:100AC0000296A11DB11D8093560290935702A093E8
:100AD0005802B0935902BF91AF919F918F910F909F
:100AE0000FBE0F901F901895AC0180E090E060E081
:100AF00020E030E0FA01E20FF31F0190F081E02DD9
:100B0000309719F08E0F9F1F6F5F2E5F3F4F203180
:100B1000310581F7772767FD70950E947411CB012D
:100B20000895FC01E55BFF4F6081718180EB94E0EB
:100B30000E947411262F862F6AE00E946811382FB8
:100B40003295307F822F0E946811832F890F08957C
:100B5000FC018FB7F8948FBF7894EC5BFF4F8091C6
:100B6000560290915702A0915802B0915902808389
:100B70009183A283B38312921292E054F04080E4F6
:100B800011928A95E9F70895CF93DF93EC016623DC
:100B900091F4C15BDF4F8881CF54D0408823F9F4B2
:100BA00083E10E94E50B892BD1F08881998160E077
:100BB00071E00E94960DC05BDF4F21E028832597EE
:100BC00088E893E19983888324962883CF54D04082
:100BD000CE010E94A80581E0DF91CF91089583E1C5
:100BE0000E94E50BC15BDF4F888380E0F5CF0F9358
:100BF0001F938C01FC018081918169E171E00E9469
:100C0000960DF8018081918164E271E00E94960D59
:100C1000F8018081918161E371E00E94960DF801F5
:100C20008081918160E471E00E94960DF8018081DD
:100C3000918162E571E00E94960DF80180819181B9
:100C400061E671E00E946B0CC8010E94A8051F912B
:100C50000F9108950F931F93CF93DF93EC011092A0
:100C6000330210924402CE5BDF4F5881C254D04011
:100C7000DE0190E030E020E021C012968C911297C6
:100C800013964C91139780FD17C0933011F0973055
:100C900051F4E22FF0E0EE0FFF1FEC5CFD4F80837C
:100CA00041832F5F09C0E32FF0E0EE0FFF1FEB5BE6
:100CB000FD4F808341833F5F9F5F12965917ECF68B
:100CC00030934402209333028881998165E671E074
:100CD0000E946B0C84E392E00E947405BC01C55B2A
:100CE000DF4F99838883CB54D040888199814AE033
:100CF00050E00E947D0D8881998164E771E00E9437
:100D00006B0C0881198185E492E00E947405BC0196
:100D1000C8014AE050E00E947D0D85E492E00E9407
:100D20007405C35BDF4F9983888323961882C0556F
:100D3000D0408881998163E871E00E94960DDF912F
:100D4000CF911F910F910895BF92CF92DF92EF92B2
:100D5000FF920F931F93DF93CF93CDB7DEB76097CA
:100D60000FB6F894DEBF0FBECDBF7B0100E010E0F0
:100D70006E010894C11CD11CF801EE0FFF1FEF5843
:100D8000FE4F65917491C6010E944403C701B601EC
:100D90000E944B03009739F00F5F1F4F0A33110574
:100DA00059F78FE307C0E02FFF27E7FDF095EB51E0
:100DB000FE4F849160960FB6F894DEBF0FBECDBF94
:100DC000CF91DF911F910F91FF90EF90DF90CF9027
:100DD000BF9008952F923F924F925F926F927F92B1
:100DE0008F929F92AF92BF92CF92DF92EF92FF923B
:100DF0000F931F93DF93CF93CDB7DEB763970FB6F3
:100E0000F894DEBF0FBECDBF7C01FE01319680E1BC
:100E1000DF011D928A95E9F722E430E0E20EF31E2D
:100E2000D701BC91B98B2EEB3FEFE20EF31E509031
:100E3000440260903302470177244424C701855B54
:100E40009F4F9B8B8A8B9DE4292E312C2E0C3F1CAF
:100E500067C0D40112960D911C91139700FD5BC0E1
:100E6000B80180E090E00E9434105B016C01EA89D7
:100E7000FB896081718180E090E00E94341020E065
:100E800030E040EC5FE30E94E6109B01AC01C6013C
:100E9000B5010E9430108823ACF4E1E0F0E0EC0FE3
:100EA000FD1FE70DF11D2EE220837394E62DF0E087
:100EB000EE0FFF1FEC5CFD4F11830083639437E05E
:100EC000632229C0D1016D917C9180E090E00E9465
:100ED000341020E030E040EC5FE30E94E6109B011C
:100EE000AC01C601B5010E9430108823A4F4E1E0F2
:100EF000F0E0EC0FFD1FE70DF11DBDE2B083739430
:100F0000E52DF0E0EE0FFF1FEB5BFD4F118300833B
:100F10005394E7E05E22439422E030E0820E931E79
:100F2000398943160CF495CF5092440260923302F3
:100F3000C701BE016F5F7F4F0E94A406182F84E394
:100F400092E00E947405ABE4B0E0EA0EFB1EF701EC
:100F5000819391937F0185E492E00E947405F701EB
:100F600091838083812F63960FB6F894DEBF0FBE06
:100F7000CDBFCF91DF911F910F91FF90EF90DF9048
:100F8000CF90BF90AF909F908F907F906F905F9029
:100F90004F903F902F9008951F93CF93DF93EC01D4
:100FA0008AE292E060E070E00E945403893611F01A
:100FB00080E03AC08AE292E062E070E00E9454036E
:100FC000182F8AE292E061E070E00E945403C55B52
:100FD000DF4F312F20E090E0282B392B29933993D4
:100FE0008AE292E064E070E00E945403182F8AE2E3
:100FF00092E063E070E00E945403312F20E090E023
:10100000282B392B398328838AE292E065E070E04F
:101010000E945403259789938AE292E066E070E08B
:101020000E945403888381E0DF91CF911F9108953E
:10103000CF92DF92EF92FF920F931F938C014AE2BF
:10104000E42E42E0F42EC70160E070E049E60E9421
:101050005B033BE4C32ED12CC00ED11EC70161E05F
:1010600070E0F60140810E945B03F6014181C701F7
:1010700062E070E00E945B032DE4C22ED12CC00E12
:10108000D11EC70163E070E0F60140810E945B035E
:10109000F6014181C70164E070E00E945B03085BD8
:1010A0001F4FC70165E070E0F80141918F010E9478
:1010B0005B03C70166E070E0F80140810E945B03BA
:1010C0001F910F91FF90EF90DF90CF900895EF92D6
:1010D000FF920F931F93CF93DF93EC0160E00E9488
:1010E000C405882309F0E1C082E10E94E50BF82ED7
:1010F0008FB7F8948FBF7894CC5BDF4F0091560286
:101100001091570288819981C454D040081B190B53
:101110000A30110508F46CC1C75BDF4F8881C954E0
:10112000D040882361F0FF2051F081E164EF71E04D
:1011300020E030E040E050E00E94130E03C081E167
:101140000E94F50DCD5BDF4F8881C354D040F81667
:1011500009F0F7C0C55BDF4F28813981CB54D040FF
:10116000C901880F991F820F931F0817190708F4E8
:101170003FC1FF2009F03CC1CE5BDF4F8881C254E4
:10118000D040882309F434C1CE010E94EA06082F1A
:1011900070E5E72EF12CEC0EFD1EF701808188230F
:1011A00009F056C0073039F482E08083CE010E94F6
:1011B000F7058BEB1EC1C85BDF4F8881C854D04058
:1011C000882389F5909155029E3269F4888199812E
:1011D00060E240E050E00E94520D802F81568A313B
:1011E00010F5005220C0C65BDF4F8881CA54D04042
:1011F0008823C9F09830B9F09A30A9F00C3299F0F0
:101200000D322CF4083079F00A3019F40CC00E328B
:1012100051F08881998160E240E050E00E94520DD7
:10122000CE010E94180888819981602F40E050E02B
:101230000E94520DC65BDF4F1882CA54D040009303
:101240005502CE010E94A805CE010E949105D1C091
:10125000823009F072C00233F1F0033324F4013319
:1012600009F05CC006C0033311F1043309F056C025
:101270003AC08881998163EA71E00E94960DF70176
:101280001082CE010E941808CE010E94A805CE014E
:101290000E949105AEC08881998160E071E00E9452
:1012A000960DCE0161E00E94C4058AEAA2C0C85B27
:1012B000DF4F8881C854D040882311F080E001C0FE
:1012C00082E08E01085B1F4FF8018083888199813D
:1012D0006CEC71E00E946B0C28813981F8018081EF
:1012E0008823C1F014C08E01075B1F4F81E0F80115
:1012F0009081891B80838881998160EE71E00E94D2
:101300006B0C28813981F8018081882319F469EDFB
:1013100071E002C06DED71E0C90104C0888199815E
:101320006AEE71E00E94960D8881998161E671E014
:101330000E946B0CCE010E941808CE010E94A805E5
:1013400057C0F1E0FF1681F4C35BDF4F88819981BC
:10135000CD54D040880F991F8017910728F4C65BA1
:10136000DF4FF882CA54D0408FB7F8948FBF78947B
:10137000CC5BDF4F8091560290915702A0915802AA
:10138000B091590288839983AA83BB83FA922A91E8
:10139000C254D040E22FFF27E7FDF0953196EE0FC3
:1013A000FF1FEC0FFD1F8F2D992787FD90950E7F56
:1013B000800F911F91838083C05BDF4F8881C05570
:1013C000D040813061F4293054F0CE010E942A06C9
:1013D000CE010E94A805CE010E9491050AC0FE011F
:1013E000EE5BFF4F80818F5F808385310CF0108230
:1013F00080E0DF91CF911F910F91FF90EF900895C2
:101400001F93CF93DF93EC017983688382E160E0DF
:101410000E94780B83E160E00E94780B83E161E039
:101420000E94980B81E161E00E94780BC15BDF4F65
:1014300011E01883CF54D040CE010E94A805C85BAC
:10144000DF4F1882239619921992198218822497D5
:10145000199310925602109257021092580210924D
:101460005902109255021882CA54D040CE010E94EF
:10147000CC07882329F4CE0161E00E94C40503C093
:10148000C05BDF4F188280916E0010926E008091D9
:101490006F00816080936F00DF91CF911F9108955D
:1014A0008AE592E060E372E00E94000A08950F93DB
:1014B0001F93CF93DF938C01C0E0D0E005C088EE8E
:1014C00093E00E94340B2196C017D107C0F3DF913F
:1014D000CF911F910F910895CF93DF9380916E006C
:1014E00010926E0080916F00816080936F008091F8
:1014F0000D0261E00E94780B80910E0261E00E9473
:10150000780BC6E0D2E0899161E00E94780B82E01E
:10151000CD30D807C1F71092AE0280E48093AB02C1
:101520008093AC02DF91CF9108951F93CF93DF9307
:10153000E091AD02F0E0E555FD4F1081C6E0D2E04C
:10154000612F617089910E94980B169582E0CD30D1
:10155000D807B1F780910D0261E00E94980B80914D
:101560000E0261E00E94980BE091AD02F0E0E35FB3
:10157000FD4F808160E00E94980B8AE090E00E941D
:10158000570A81E09091AD02891B8093AD02DF91F3
:10159000CF911F91089580E392E00E94E7040E949A
:1015A000950A8AE592E00E9467088823A1F0A82F97
:1015B000B0E0FD0184E0F595E7958A95E1F7E15FFC
:1015C000FD4F80818093AB02AF70B070A15FBD4FC3
:1015D0008C918093AC0208951F920F920FB60F92D8
:1015E00011242F933F938F939F93AF93BF93809139
:1015F000B3029091B402A091B502B091B6023091BD
:10160000B7020196A11DB11D232F2D5F2D3720F0AC
:101610002D570196A11DB11D2093B7028093B302EF
:101620009093B402A093B502B093B6028091AF023A
:101630009091B002A091B102B091B2020196A11DA9
:10164000B11D8093AF029093B002A093B102B0930A
:10165000B202BF91AF919F918F913F912F910F90C7
:101660000FBE0F901F901895019739F0880F991FA2
:10167000880F991F02970197F1F70895789484B520
:10168000826084BD84B5816084BD85B5826085BD7E
:1016900085B5816085BDEEE6F0E080818160808364
:1016A000E1E8F0E0808182608083808181608083D6
:1016B000E0E8F0E0808181608083E1EBF0E0808110
:1016C00084608083E0EBF0E0808181608083EAE7E2
:1016D000F0E080818460808380818260808380816B
:1016E000816080838081806880831092C10008952A
:1016F000282F30E0C9018C569C4FFC019491205852
:101700003C4FF9018491882391F0E82FF0E0EE0F2F
:10171000FF1FEE59FC4FA591B491662329F48C91DB
:10172000909589238C9308958C91892B8C9308959F
:10173000482F50E0CA0188559C4FFC012491CA01F2
:101740008C569C4FFC01949140585C4FFA013491A7
:101750003323D1F1222331F1233021F48091800011
:101760008F7705C0243031F4809180008F7D809385
:10177000800018C0213019F484B58F7704C022305E
:1017800021F484B58F7D84BD0DC0263021F4809175
:10179000B0008F7705C0273029F48091B0008F7D8D
:1017A0008093B000E32FF0E0EE0FFF1FE459FC4FF1
:1017B000A591B491662329F48C91909589238C93FB
:1017C00008958C91892B8C930895682F70E0CB013C
:1017D00088559C4FFC012491CB018C569C4FFC01F9
:1017E000449160587C4FFB019491992319F420E0B7
:1017F00030E038C0222331F1233021F48091800081
:101800008F7705C0243031F4809180008F7D8093E4
:10181000800018C0213019F484B58F7704C02230BD
:1018200021F484B58F7D84BD0DC0263021F48091D4
:10183000B0008F7705C0273029F48091B0008F7DEC
:101840008093B000892F90E0880F991F8A589C4F91
:10185000FC01A591B4918C9120E030E0842311F03B
:1018600021E030E0C90108950F931F93CF93DF93D8
:101870008C01EB0109C02196D801ED91FC910190FA
:10188000F081E02DC801099568816623A1F7DF91F9
:10189000CF911F910F910895EF92FF920F931F9395
:1018A000CF93DF938C017B01EA010CC0D7016D91CE
:1018B0007D01D801ED91FC910190F081E02DC801EE
:1018C00009952197209791F7DF91CF911F910F9163
:1018D000FF90EF900895DC01ED91FC910280F3817F
:1018E000E02D099508952F923F924F925F926F924B
:1018F0007F928F929F92AF92BF92CF92DF92EF92A0
:10190000FF920F931F93DF93CF93CDB7DEB7A097CE
:101910000FB6F894DEBF0FBECDBF1C016A017B017C
:10192000411551056105710549F440E350E060E05F
:1019300070E020E030E00E941C0D56C088249924FD
:101940005401422E55246624772401E010E00C0F48
:101950001D1F080D191DC701B601A30192010E94A8
:101960008811F80160830894811C911CA11CB11C92
:10197000C701B601A30192010E948811C901DA01D1
:101980006C017D01C114D104E104F104F1F681E0A0
:10199000E82EF12CEC0EFD1EE80CF91C3E0108941B
:1019A000611C711CD501C4010197A109B1096C0129
:1019B000C818D90816C0F601EE0DFF1D40814A3047
:1019C00010F4405D01C0495C552747FD5095652FD7
:1019D000752FC10120E030E00E941C0D0894E10841
:1019E000F1086E147F0439F7A0960FB6F894DEBFA5
:1019F0000FBECDBFCF91DF911F910F91FF90EF9060
:101A0000DF90CF90BF90AF909F908F907F906F901E
:101A10005F904F903F902F900895DC012115310584
:101A200041F4ED91FC910190F081E02D642F099536
:101A300008950E94730C0895EF92FF920F931F93E5
:101A4000CF93DF93EC017A018B012115310541F42D
:101A5000E881F9810190F081E02D642F09951BC088
:101A60002A303105B1F477FF10C04DE250E060E05C
:101A700070E020E030E00E941C0D10950095F0947D
:101A8000E094E11CF11C011D111DCE01B801A7015C
:101A90002AE00E94730CDF91CF911F910F91FF906C
:101AA000EF900895EF92FF920F931F93E62E9A0105
:101AB000FF24E7FCF0940F2D1F2DB801A7010E9411
:101AC0001C0D1F910F91FF90EF9008950F931F939E
:101AD0008C014DE050E060E070E020E030E00E94DA
:101AE0001C0DC8014AE050E060E070E020E030E00A
:101AF0000E941C0D1F910F910895CF92DF92EF92DB
:101B0000FF920F931F938C019A016B01EE24FF2427
:101B1000B701A6010E940D0DC8010E94660D1F911C
:101B20000F91FF90EF90DF90CF9008950F931F9348
:101B30008C010E946B0CC8010E94660D1F910F91D1
:101B400008951F920F920FB60F9211248F939F93B7
:101B5000AF93BF93EF93FF938091C6029091C7021A
:101B6000A091C802B091C902E091CA02F091CB02E3
:101B70000097A105B10531F180819091CC028927B0
:101B800080838091C6029091C702A091C802B09153
:101B9000C902181619061A061B06E4F48091C6023B
:101BA0009091C702A091C802B091C9020197A10902
:101BB000B1098093C6029093C702A093C802B09364
:101BC000C90208C01092700090818091CC0280956B
:101BD00089238083FF91EF91BF91AF919F918F9166
:101BE0000F900FBE0F901F901895282F80911F0205
:101BF0008217A1F4E1E6F3E094918FEF80931F0246
:101C0000913039F0923041F0992341F410926E00F6
:101C100005C010926F0002C010927000822F60E029
:101C20000E94980B08952F923F925F926F927F923D
:101C30008F929F92AF92BF92CF92DF92EF92FF92DC
:101C40000F931F93DF93CF9300D000D0CDB7DEB7B3
:101C5000A82F1B0129833A834B835C8380911F0249
:101C60008A1721F4E1E6F3E0549082C08F3F09F037
:101C7000DAC1A0931F02E1E6F3E054902FEF521671
:101C800009F4D1C181E0581639F192E0591609F4EE
:101C900049C0552009F06CC014BC15BC84B58260E5
:101CA00084BD85B5816085BD2A2F30E0F901E058FB
:101CB000FC4FE491F0E0EE0FFF1FE459FC4F8591DB
:101CC00094919093BD028093BC022C563C4FF90135
:101CD00084918093BE024EC01092800010928100C9
:101CE0008091810088608093810080918100816073
:101CF000809381002A2F30E0F901E058FC4FE491F5
:101D0000F0E0EE0FFF1FE459FC4F85919491909302
:101D1000C4028093C3022C563C4FF90184918093F6
:101D2000C50228C01092B0001092B1008091B0009E
:101D300082608093B0008091B10081608093B10097
:101D40002A2F30E0F901E058FC4FE491F0E0EE0F6B
:101D5000FF1FE459FC4F859194919093CB0280939F
:101D6000CA022C563C4FF90184918093CC0202C0E8
:101D700057FC59C18A2F61E00E94780B552021F051
:101D8000F2E05F1609F0BEC031018824992460E0BA
:101D900072E18AE790E0A40193010E94AA1159011F
:101DA0006A01860175010894E108F1080109110929
:101DB0002FEFE216F1040105110509F008F499C0AE
:101DC00060E472E48FE090E0A40193010E94AA1104
:101DD00079018A010894E108F1080109110982E0FA
:101DE0005816C1F49FEFE916F1040105110509F039
:101DF00008F484C060E970ED83E090E0A4019301F1
:101E00000E94AA1179018A010894E108F1080109E8
:101E1000110983E0AFEFEA16F1040105110509F09D
:101E200008F468C068E478EE81E090E0A4019301D2
:101E30000E94AA1179018A010894E108F1080109B8
:101E40001109552011F483E01DC0B2E05B1611F0BA
:101E500084E018C0EFEFEE16F1040105110509F05A
:101E600008F4DFC064E274EF80E090E0A401930125
:101E70000E94AA1179018A010894E108F108010978
:101E8000110985E0FFEFEF16F1040105110591F14D
:101E900088F162E17AE780E090E0A40193010E947A
:101EA000AA1179018A010894E108F10801091109D0
:101EB000552011F086E001C084E02FEFE216F10416
:101EC00001051105B9F0B0F0C601B50120E034E01C
:101ED00040E050E00E94AA1179018A010894E108CB
:101EE000F10801091109552011F087E008C085E0CB
:101EF00003C081E0552019F485BD3AC082E080938B
:101F0000B10036C05101CC24DD2460E072E18AE7E3
:101F100090E0A60195010E94AA1179018A01089416
:101F2000E108F1080109110980E0E81680E0F806EF
:101F300081E0080780E0180710F491E010C068E421
:101F400078EE81E090E0A60195010E94AA11790146
:101F50008A010894E108F1080109110993E0A1E060
:101F60005A1631F480918100887F982B90938100DC
:101F700089819A81AB81BC810097A105B10529F4C3
:101F80008FEF9FEFAFEFBFEF13C0220C331CB101F7
:101F900080E090E029813A814B815C810E94491167
:101FA00028EE33E040E050E00E948811C901DA01D8
:101FB000E1E05E16A1F0F2E05F1619F1552099F507
:101FC000E7BC8093B8029093B902A093BA02B09391
:101FD000BB0280916E00826080936E0024C0F092FC
:101FE0008900E09288008093BF029093C002A09382
:101FF000C102B093C20280916F00826080936F0033
:1020000012C0E092B3008093C6029093C702A093DF
:10201000C802B093C9028091700082608093700002
:1020200002C084E06CCF0F900F900F900F90CF9173
:10203000DF911F910F91FF90EF90DF90CF90BF90B5
:10204000AF909F908F907F906F905F903F902F9078
:1020500008950E943E0B0E946C0A0E94CB0AFDCF9D
:1020600040D008F481E00895E89409C097FB3EF45D
:1020700090958095709561957F4F8F4F9F4F9923D5
:10208000A9F0F92F96E9BB279395F6958795779553
:102090006795B795F111F8CFFAF4BB0F11F460FF13
:1020A0001BC06F5F7F4F8F4F9F4F16C0882311F06B
:1020B00096E911C0772321F09EE8872F762F05C07F
:1020C000662371F096E8862F70E060E02AF09A951A
:1020D000660F771F881FDAF7880F9695879597F90F
:1020E0000895990F0008550FAA0BE0E8FEEF1616A9
:1020F0001706E807F907C0F012161306E407F507FC
:1021000098F0621B730B840B950B39F40A2661F06F
:10211000232B242B252B21F408950A2609F4A14012
:10212000A6958FEF811D811D089597F99F6780E81F
:1021300070E060E008959FEF80EC089500240A9419
:102140001616170618060906089500240A94121692
:102150001306140605060895092E0394000C11F4C5
:10216000882352F0BB0F40F4BF2B11F460FF04C072
:102170006F5F7F4F8F4F9F4F089557FD9058440FCB
:10218000551F59F05F3F71F04795880F97FB991FD6
:1021900061F09F3F79F08795089512161306140693
:1021A000551FF2CF4695F1DF08C016161706180620
:1021B000991FF1CF86957105610508940895E894FB
:1021C000BB2766277727CB0197F908950BD0C4CF9B
:1021D000B5DF28F0BADF18F0952309F0A6CFABCF12
:1021E0001124EECFCADFA0F3959FD1F3950F50E0F5
:1021F000551F629FF001729FBB27F00DB11D639FB9
:10220000AA27F00DB11DAA1F649F6627B00DA11D5E
:10221000661F829F2227B00DA11D621F739FB00D04
:10222000A11D621F839FA00D611D221F749F332774
:10223000A00D611D231F849F600D211D822F762F0D
:102240006A2F11249F5750408AF0E1F088234AF00A
:10225000EE0FFF1FBB1F661F771F881F9150504056
:10226000A9F79E3F510570F060CFAACF5F3FECF316
:10227000983EDCF3869577956795B795F795E79542
:102280009F5FC1F7FE2B880F911D9695879597F953
:102290000895629FD001739FF001829FE00DF11DB0
:1022A000649FE00DF11D929FF00D839FF00D749FD0
:1022B000F00D659FF00D9927729FB00DE11DF91F7C
:1022C000639FB00DE11DF91FBD01CF0111240895D9
:1022D000991B79E004C0991F961708F0961B881F78
:1022E0007A95C9F780950895AA1BBB1B51E107C0D9
:1022F000AA1FBB1FA617B70710F0A61BB70B881F96
:10230000991F5A95A9F780959095BC01CD01089524
:10231000A1E21A2EAA1BBB1BFD010DC0AA1FBB1FE9
:10232000EE1FFF1FA217B307E407F50720F0A21B5B
:10233000B30BE40BF50B661F771F881F991F1A94C8
:1023400069F760957095809590959B01AC01BD01F2
:10235000CF01089597FB092E05260ED057FD04D016
:10236000D7DF0AD0001C38F4509540953095219560
:102370003F4F4F4F5F4F0895F6F7909580957095BA
:1023800061957F4F8F4F9F4F0895EE0FFF1F059070
:0A239000F491E02D0994F894FFCFBA
:10239A000A4C6561726E696E672E20456E746572AD
:1023AA0020272D2E2D2E2D270053657474696E67F4
:1023BA00732E3A002020312E204E6F726D616C2EE2
:1023CA00002020322E204C6561726E696E672E00E5
:1023DA002020332E204175746F2D666F726D6174E3
:1023EA002E002020342E2053696465746F6E652E8A
:1023FA00002D3E20004176672064697420286D73A1
:10240A00293A20004176672064616820286D732983
:10241A003A2000446F6E652E2027534F53272074AD
:10242A006F20656E746572206D61696E206D656ED0
:10243A00752E004E6F726D616C206D6F64652E2073
:10244A0027534F532720746F207265656E74657227
:10245A002074686973206D656E752E004175746FFE
:10246A0020666F726D617420004F4646004F4E0021
:10247A0053696465746F6E652000556E6B6E6F7775
:10248A006E20636F64652E205472792061676169DA
:10249A006E2E20005AFF070B0C090A08060D053F8D
:1024AA00065B4F666D7D070F6F38403F5E7971FF9F
:0A24BA0000000000EA04340C4C0C92
:00000001FF
